:020000040000FA
:04000000A7EF0DF069
:08000800056ED8CF06F0E0CF31
:1000100007F00001E9CF0DF0EACF08F0E1CF09F0D9
:10002000E2CF0AF0D9CF0BF0DACF0CF0F3CF14F017
:10003000F4CF15F0FACF16F000C00FF001C010F0A9
:1000400002C011F003C012F004C013F0F2AA2CEFAA
:1000500000F0F2B4B1EF01F0A0AA32EF00F0A1BAC3
:10006000BCEF08F00FC000F010C001F011C002F0AA
:1000700012C003F013C004F00DC0E9FF08C0EAFF8E
:10008000088E09C0E1FF0AC0E2FF0BC0D9FF0CC017
:10009000DAFF14C0F3FF15C0F4FF16C0FAFF0550D5
:1000A00007C0E0FF06C0D8FF1000F2CF0EF0F29EAE
:1000B000F76AC40FF66E000EF7220900F5500EBE67
:1000C000F28E1200280C0106F76AD80FF66E000EA9
:1000D000F7220900F5501200000302FFFFFFFFFFA7
:1000E000FFFFFFFFFFFFFFFFF76AF80FF66E000E3E
:1000F000F7220900F550120000FF02FFFFFFFFFF8B
:10010000FFFFFFFFFFFFFFFFF76A180FF66E010EFC
:10011000F7220900F55012004000080040000000DE
:1001200000000000000000000000000000000000CF
:100130000000000000000000F76A480FF66E010E94
:10014000F7220900F55012004000000040000000B6
:10015000000000000000000000000000000000009F
:100160000000000000000000F76A780FF66E010E34
:10017000F7220900F5501200090243000201008035
:1001800032090400000102020100052400100104EC
:10019000240202052406000105240100010705814F
:1001A000030800FA09040100020A00000007050222
:1001B000024100010705820241000100F76ACC0FED
:1001C000F66E010EF7220900F55012000200F76AE0
:1001D000DE0FF66E010EF7220900F550120012171D
:1001E0001B20FFFFFFFFF76AF60FF66E010EF722E6
:1001F0000900F550120012011001020000406104D4
:100200003300000101020001F76A180FF66E020EBA
:10021000F7220900F5501200040309040803430003
:1002200043005300180353004500520049004100A9
:100230004C002000440045004D004F00F2CF0EF06E
:10024000F29EF76A560FF66E020EF7220900F5507D
:100250000EBEF28E12000C2053544F50574154439F
:10026000483031410000F2CF0EF0F29EF76A800F65
:10027000F66E020EF7220900F5500EBEF28E120045
:10028000204B616B6C696B20323031300000F2CF53
:100290000EF0F29EF76AA80FF66E020EF722090022
:1002A000F5500EBEF28E12000C57616974696E67CC
:1002B00020666F722050432E2E2E2000F2CF0EF0BB
:1002C000F29EF76AD60FF66E020EF7220900F5507D
:1002D0000EBEF28E12000C20504320636F6E6E65CE
:1002E000637465642E2E2E00F2CF0EF0F29EF76A34
:1002F000020FF66E030EF7220900F5500EBEF28EC5
:1003000012000C0A53544152542020202020202057
:10031000544553540000F2CF0EF0F29EF76A300FAE
:10032000F66E030EF7220900F5500EBEF28E120093
:100330000C0A202020202020202045534300F2CF0B
:100340000EF0F29EF76A580FF66E030EF7220900C0
:10035000F5500EBEF28E12000C0A20202053544F8E
:100360005000010E2926D8B02A2AD8B42B2AD8B496
:100370002C2AF29432EF00F06D92699468A402D0B6
:100380006894FCD7C7EF08F0400E0401016F040E1B
:10039000036F180E026F880E006F046B040E076F58
:1003A000580E066F0001000C70A002D0EDDF7090B7
:1003B000689AD0EF08F06A6A6892D6EF08F0DD51CB
:1003C000DF03F3CF01F0F4CF00F0E003F350002699
:1003D000DE51DF03F3500020026E000C036AD75198
:1003E000700FE96E0F0E0320EA6EEF6ADE6BD7C066
:1003F000DDF0E06B080EDF6FE2DF01C0E9FF040E05
:100400000224EA6EEF6ADE6BD7C0DDF0E06B080E07
:10041000DF6FD5DF02C0D9F001C0D8F0040ED827B5
:10042000000ED923D8C0E9FF040ED925EA6EEF6A81
:10043000000C010ED66FD6510F0805E3D6C0D7F0D9
:10044000CDDFD62BF8D7000C426A416A250E406EEC
:10045000800E3F6E436A446A080E456E956B949118
:10046000476A466A906B9191000CCC6BCC510108A5
:100470000AE3036ACC513D0FE96E000E0320EA6ED9
:10048000EF6ACC2BF3D7E0DF326A010E336E316AAC
:10049000000C689600D000D000D0000C6A6A686A30
:1004A0009F0E6B6E3D0E696E6E6AC3DFDEDF160E49
:1004B000706E68A602D0EDDFFCD76D9865DF030E85
:1004C000386EDCEF08F0698468986D82E2EF08F01E
:1004D000689CE8EF08F0D1C039F0000CFF0E396ECF
:1004E000000CCF6B3C5237E0CF513F0834E334501F
:1004F00005E0020A0DE0010A15E01ED0036A3B5038
:10050000F2CFD1F0F29E30DED1BFF28ED06F14D098
:10051000036A3B50F2CFD1F0F29E76DED1BFF28E6D
:10052000D06F0AD0036A3B50F2CFD1F0F29E5BDE6F
:10053000D1BFF28ED06F00D03B2A3C06CF51CF2BDB
:10054000580F036AD8B0032AE96E040E0324EA6E3A
:10055000D0C0EFFFC7D73C5204E1CF51400801E0C3
:10056000316ACFC0D1F0B7DF000C3B6A346A0401B6
:100570001B51010A000107E0030A0AE0010A0BE02F
:10058000220A20E03AD0120E3C6E030E346E37D0B1
:10059000430E3C6E34D0020E346E036A04011A51CD
:1005A000350FE96E000E0320EA6EEFCF3BF0036AD1
:1005B0003B50F2CFCEF0F29E000126DECEBFF28E8F
:1005C0003C6E1DD0036A04011A51F2CFCEF0F29EA8
:1005D0000001FDDDCEBFF28E3B6E3B3C01D00BD067
:1005E000036A3B50F2CFCEF0F29EBEDDCEBFF28E5C
:1005F0003C6E05D002D072DF0ED070DF0CD004014B
:100600001F5305E13C501E5D02E21EC43CF0010E8A
:10061000316E000166DF4BEF04F0CE5304E1040EAF
:10062000386E07DFE7D0050E386E040ED16F980ED6
:10063000D06F010ECF6FCF510F08D8A0DBD0CFC045
:10064000D7F0CCDED26B036ACF51F2CFD6F0F29E58
:100650004BDDD6BFF28EFF0863E0040ED26FD89058
:10066000CF35036AF2CFD6F0F29E66DD0900F5CFF2
:1006700003F0D6BFF28ED36F03C0D4F0DE6BCFC0D1
:10068000DDF0E06B080EDF6F9ADE01C0D6F0010EE0
:100690000124016E000E0220036E01C0E9FF040E6A
:1006A0000324EA6ED3C0EFFFDE6BCFC0DDF0E06B5A
:1006B000080EDF6F84DE01C0D6F0020E0124016E49
:1006C000000E0220036E01C0E9FF040E0324EA6E4F
:1006D000D1C0ECFFED52D0C0EFFFD890CF35036A08
:1006E000F2CFD6F0F29E28DD0900F5CF03F0D6BF99
:1006F000F28ED0270350D123880ED56FD4B1D58187
:10070000D4B3D583DE6BCFC0DDF0E06B080EDF6FB6
:1007100056DE01C0E9FF040E0224EA6ED5C0EFFFE9
:10072000036ACF51F2CFD6F0F29ECEDCD6BFF28E66
:10073000FF0845E0D283DE6BCFC0DDF0E06B080E32
:10074000DF6F3DDE02C0D7F001C0D6F0040ED62721
:10075000000ED723020ED625016E000ED721036EA0
:1007600001C0E9FF040E0324EA6ED1C0ECFFED5294
:10077000D0C0EFFFD890CF35036AF2CFD6F0F29E0B
:10078000C3DC0900F5CF03F0D6BFF28ED0270350AB
:10079000D123DE6BCFC0DDF0E06B080EDF6F0FDE24
:1007A00002C0D7F001C0D6F0040ED627000ED72322
:1007B000D6C0E9FF040ED725EA6E400EEF6ED25187
:1007C000060802E10E0ED26F036ACF51F2CFD6F0C7
:1007D000F29E7ADCD6BFF28E0108D8A4D289036AD1
:1007E000CF51700FE96E0F0E0320EA6ED2C0EFFFFB
:1007F000CF2B21D745EF04F00401195100010DE082
:10080000010A14E0020A1EE0060A27E0030A2CE0AF
:100810000E0A2BE0010A2FE03CD033C058F404014B
:10082000596B020E0001D16F56DE35D004011A2D2E
:1008300006D0010E33160001D16B4DDE02D000014F
:100840004DDE29D004011A2D05D033820001D16B71
:1008500042DE02D0000142DE1ED0020E316E1AC40A
:100860003AF0D16B38DE17D080D632C058F4010E82
:10087000D16F31DE10D004011A51010808E31AC407
:1008800032F01AC4CEF00001C8D6D16B24DE0001CC
:1008900002D024DE00D0E6EF05F032C0CEF0040135
:1008A0001951000105E00A0A0BE0010A2BE03CD0D7
:1008B0000401586B596B020E0001D16F0CDE36D06B
:1008C000CE531EE0010ECE5D036AF2CFCFF0F29E52
:1008D00075DCCFBFF28E016E04011C5DD8A002D082
:1008E00000010ED0036A1C513D0FE96E000E03207B
:1008F000EA6EEFCF58F4010E0001D16FECDD01D0AC
:10090000EDDD14D0CE530EE0036A04011C513D0FFF
:10091000E96E000E0320EA6E1AC4EFFF0001D16BEE
:10092000DADD01D0DBDD02D0D9DD00D0E6EF05F065
:10093000CF91CEBFCF81CE9FCFA111D0036ACE5130
:10094000F2CFD0F0F29E64EC00F0D0BFF28EFF0840
:1009500002E1000E01D0010E016E11D010D0036A29
:10096000CE51F2CFD0F0F29E74EC00F0D0BFF28EF8
:10097000FF0802E1000E01D0010E016E00D052EF1F
:1009800005F0CF91CEBFCF81CE9FCFA117D0DE6B28
:10099000CEC0DDF0E06B080EDF6F11DD02C0D1F0DC
:1009A00001C0D0F0040ED027000ED123D0C0E9FF43
:1009B000040ED125EA6E880EEF6E0DD0DE6BCEC030
:1009C000DDF0E06B080EDF6FFADC01C0E9FF040E1A
:1009D0000224EA6EEF6A61EF05F0CF91CEBFCF81BE
:1009E000CE9FCFA117D0DE6BCEC0DDF0E06B080E3E
:1009F000DF6FE5DC02C0D1F001C0D0F0040ED027DB
:100A0000000ED123D0C0E9FF040ED125EA6E840E7A
:100A1000EF6E0ED0DE6BCEC0DDF0E06B080EDF6F48
:100A2000CEDC01C0E9FF040E0224EA6E840EEF6EF4
:100A300067EF05F0CF91CEBFCF81CE9FCFA117D06A
:100A4000DE6BCEC0DDF0E06B080EDF6FB8DC02C0FD
:100A5000D2F001C0D1F0040ED127000ED223D1C0B4
:100A6000E9FF040ED225EA6EEFCFD0F00ED0DE6B98
:100A7000CEC0DDF0E06B080EDF6FA1DC01C0E9FF46
:100A8000040E0224EA6EEFCFD0F0D0AF02D0D0B582
:100A900002D0000E01D0010E016E71EF05F01CC4F2
:100AA000CEF046D7015229E004011951010A000194
:100AB00005E0020A09E0030A0DE01DD01CC4CEF0D7
:100AC00060D7D16B08DD19D01CC4CEF086D7D16BAE
:100AD00002DD13D00401586B596B1CC4CEF0000129
:100AE000A9D7015204E0010E0401586F0001020E63
:100AF000D16FF1DC02D0F2DC00D0E6EF05F0FE0EA3
:100B0000396E000C04011C2D01D002D01C5348E1A9
:100B1000195100010BE0010A0DE0210A1CE0010A55
:100B20001FE0030A2EE0010A31E037D0010E976F73
:100B3000E6DF35D0040EEA6E580EE96EE26A480E22
:100B4000E16E080E016EE6CFEEFF012EFCD71EC44B
:100B5000D1F0C1DC24D0020E976F9481D0DF1FD07A
:100B6000040EEA6E580EE96EE26A3F0EE16E070E61
:100B7000016EE6CFEEFF012EFCD7070ED16FABDC86
:100B80000ED01AC495F0D16BA6DC09D01AC447F078
:100B90001BC446F0D16B9FDC02D0A0DC00D0040166
:100BA0000001E6EF05F0316A040118517F0B0001E6
:100BB00007E0010A06E0030A05E0230A04E004D086
:100BC0001BD66BD66CD79ED789DC00D00AEF08F015
:100BD000DE6BCEC0DDF0E06B080EDF6FDFEC01F006
:100BE00001C0E9FF040E0224EA6EEFCFD0F0CF512E
:100BF000020806E1D0AD02D0CF6B02D0010ECF6F5C
:100C0000CF5103081AE1840ED06FDE6BCEC0DDF049
:100C1000E06B080EDF6FDFEC01F002C0D4F001C022
:100C2000D3F0040ED327000ED423D3C0E9FF040E63
:100C3000D425EA6E840EEF6E07D0CF2D03D0C80EF8
:100C4000D06F02D0880ED06FD890CE35036AF2CF25
:100C5000D3F0F29E9CEC00F00900F5CF03F0D3BF77
:100C6000F28ED16F03C0D2F0DE6BCEC0DDF0E06B50
:100C7000080EDF6FDFEC01F001C0D3F0010E01249C
:100C8000016E000E0220036E01C0E9FF040E032472
:100C9000EA6ED1C0EFFFD2B1D081D2B3D083DE6B88
:100CA000CEC0DDF0E06B080EDF6FDFEC01F001C0BD
:100CB000E9FF040E0224EA6ED0C0EFFF000C036AC5
:100CC000DC51700FE96E0F0E0320EA6EEF5219E04F
:100CD000DE6BDCC0DDF0E06B080EDF6FDFEC01F0F7
:100CE00002C0DEF001C0DDF0040EDD27000EDE23C1
:100CF000DDC0E9FF040EDE25EA6EEFCFDDF0DDAFEB
:100D000002D0000E01D0010E016E000CD7C0DCF045
:100D1000D6DF0152D8B47CD0DE6BD7C0DDF0E06BFB
:100D2000080EDF6FDFEC01F002C0DDF001C0DCF087
:100D3000040EDC27000EDD23010EDC25016E000E03
:100D4000DD21036E01C0E9FF040E0324EA6ED8C062
:100D5000EFFFDA5102081EE1DE6BD7C0DDF0E06B79
:100D6000080EDF6FDFEC01F002C0DDF001C0DCF047
:100D7000040EDC27000EDD23DCC0E9FF040EDD25B8
:100D8000EA6EEFCFDBF0DBAD02D0DA6B02D0010E02
:100D9000DA6F18D0DA51040815E1DE6BD7C0DDF048
:100DA000E06B080EDF6FDFEC01F001C0E9FF040E1D
:100DB0000224EA6EEFCFDBF0DBAD03D0010EDA6F79
:100DC00001D0DA6BDA2D03D0C80EDB6F02D0880EAB
:100DD000DB6FD9B1DB81D9B3DB83DE6BD7C0DDF04C
:100DE000E06B080EDF6FDFEC01F002C0DDF001C048
:100DF000DCF0040EDC27000EDD23DCC0E9FF040E6E
:100E0000DD25EA6EDBC0EFFF010E016E03D000D0DE
:100E1000000E016E000C9751010A03E0030A13E073
:100E200024D0EA6A480EE96E040EE26E180EE16EF6
:100E3000080E016EE6CFEEFF012EFCD7D16B6BECF6
:100E400002F0976B16D0EA6A3F0EE96E040EE26E6E
:100E5000180EE16E070E016EE6CFEEFF012EFCD7F5
:100E6000976BD16B6BEC02F004D0976BC4EC01F084
:100E700000D065EF07F0DE6BCFC0DDF0E06B080E51
:100E8000DF6FDFEC01F002C0D1F001C0D0F0010E45
:100E90000124016E000E0220036E01C0E9FF040E62
:100EA0000324EA6E036AEFCF01F003C002F05EEFA5
:100EB00007F09181936B020ECF6FDDD701C092F0E6
:100EC0006AEF07F0CE5302E1A6D704D0CE51020854
:100ED00001E1EFD7000CCFC06EFFCF5303E0040E4B
:100EE000386E02D0020E386E7BEF07F0326A316A3C
:100EF0003AC0CFF0F0D7EAEF07F0CFC0DCF0DFDE8A
:100F0000015246E0DE6BCFC0DDF0E06B080EDF6F14
:100F1000DFEC01F002C0D8F001C0D7F0040ED727F3
:100F2000000ED823020ED725016E000ED821036EC5
:100F300001C0E9FF040E0324EA6EECCF03F0ED528A
:100F4000EFCFD5F003C0D6F0D6C0EAFFD5C0E9FF99
:100F5000D1C0E2FFD0C0E1FFD3C002F0D2C001F0A7
:100F6000015202E0022A02D0025206E0E6CFEEFF72
:100F7000012EFCD7022EFAD7CFC0D7F0D3C0D9F0BC
:100F8000D2C0D8F0D4C0DAF0C1DE015003D000D016
:100F9000000E016E000C020ECF6FD16B500ED06FA1
:100FA000D36B90C0D2F0020ED46FA7DF90C096F042
:100FB000906B000C905301E0EEDFEFEF07F0CE53A3
:100FC0000AE1312C03D071EC02F004D03150020858
:100FD00001E18CD704D0CE51020801E1EBD7000C1F
:100FE0006C30CC6FCC33CC331F0ECC176C5240E13D
:100FF000040100513C0B0001CD6F430E04010017AA
:10100000000149EC02F0CD5134081BE10401046BEE
:101010000001C9D56D98393C05D0CE6B030ECF6F5A
:10102000D7DD0ED0CE6B020ECF6FD2DD3950FE0869
:1010300007E0D76BD96B39C0D8F0040EDA6F66DEE3
:1010400016D0CD51040813E1CE6B3CDFCE6B020EFF
:10105000CF6FBEDD3950FE080AE0393C01D007D021
:10106000D76BD96B39C0D8F0010EDA6F4FDE82D062
:101070006C50040818E1430E04010417000149EC08
:1010800002F0FF0E396ECE6B9ADF393C01D008D0EA
:10109000D76BD96B39C0D8F0020EDA6F37DE02D0C9
:1010A000C4EC01F067D06CB42CD0DE6BCCC0DDF0AA
:1010B000E06B080EDF6FDFEC01F001C0CEF001C085
:1010C00001F0040E0224036E01C0CEF0CF6FDE6B80
:1010D000CCC0DDF0E06B080EDF6FDFEC01F001C08B
:1010E000E9FF040E0224EA6EEF50430BCFC0EAFF83
:1010F000CEC0E9FFEF6E49EC02F0CCC0CEF0E2DEEC
:1011000039D0DE6BCCC0DDF0E06B080EDF6FDFECBA
:1011100001F002C0CFF001C0CEF0040ECE27000EC9
:10112000CF23CEC001F0040ECF25036ECEC0CEF08B
:10113000CF6FDE6BCCC0DDF0E06B080EDF6FDFEC55
:1011400001F002C0D1F001C0D0F0040ED027000E93
:10115000D123D0C0E9FF040ED125EA6EEF50430B36
:10116000CFC0EAFFCEC0E9FFEF6E49EC02F0CCC081
:10117000CEF025DFEEEF08F0385201E135D06852AD
:1011800033E068A404D069A402D0BCEF01F06DA2E2
:1011900001D02AD068AA04D069AA02D0D4EF01F005
:1011A00068A204D069A202D0DBEF01F068A004D0ED
:1011B00069A002D04EEF02F068A804D069A802D05E
:1011C00063EF02F068AC04D069AC02D068EF02F0C3
:1011D000CB6B68A604D069A602D002D701D004D098
:1011E000CB51CB2B0308F5E2A19A32EF00F0EA6A6B
:1011F000A30EE96EEF500EE0070E016E006A002E9E
:10120000FED7012EFBD7C70E006E002EFED70000C2
:10121000EF2EF2D7000CAAB102D08C9801D08C88A6
:101220009598AAB302D08C9A01D08C8A959AAAB5C7
:1012300002D08C9C01D08C8C959CAAB702D08C9E3D
:1012400001D08C8E959E00008D809690030E006ECE
:10125000002EFED700D08D909690000CAB6B958839
:10126000000E83B8010EAB13958A000E83BA010EEF
:10127000006ED89000360050AB13958C000E83BCE6
:10128000010E006E00360036FC0E00160050AB1347
:10129000958E000E83BE010E006E003600360036BD
:1012A000F80E00160050AB13ABC001F0000C95888F
:1012B000958A958C958E8D84969400008D8096905D
:1012C0000000CCDF01C0AAF08D90969000008D80C8
:1012D000969000D000D000D0C1DF01C0A9F08D9061
:1012E00096909598959A959C959EAA39006EF00EC9
:1012F00000160050A911016E81EF09F08D929692AF
:10130000D6D701C0A9F001BEFBD7A75302E18D9249
:1013100001D08D82969200008D94969400008D905D
:101320009690A839A96F0F0EA917A9C0AAF073DF6C
:10133000A8510F0BA96FAA6F6EDF000C9598959AB4
:10134000959C959E9690969296948D9296928D9459
:1013500096948D9096900F0EA36F49DF010E986FB3
:101360009851030808E3030EAA6F55DF050EA36F1B
:101370003EDF982BF5D7020EAA6F4DDF986B985180
:1013800003080FE3036A9851F2CF99F0F29E55ECEF
:1013900000F099BFF28E996FA76BA86FAFDF982B03
:1013A000EED7E4EF0DF06D6A696A080E6F6E945027
:1013B0003009946E386A186AF2BE188EF29E35ECC7
:1013C00002F018BEF28EE6EF09F0EDD70CEF0AF04E
:1013D000186AF2BE188EF29E35EC02F018BEF28E3C
:1013E0006D6A140E6F6E696A6D86010E386EFCEFC1
:1013F00009F06DB601D0ECD7382C0BD06DBA09D0FE
:10140000686A696AA08AC00EF212110E696E020E35
:10141000386E0DEF0AF0D9D7ECD738500208FCE14E
:10142000E5EF0DF0A42D01D003D0400EA56F01D043
:10143000A56B010EA35DA527A5518009A66FA76B1B
:10144000A86F5CDF000CA2510C0A05E0060A0BE055
:10145000020A0FE013D0A76B010EA86F4FDF020E38
:10146000A36FC5DE11D0010EA36F020EA46FDADFE9
:101470000BD0A76B100EA86F41DF06D0010EA76F2F
:10148000A2C0A8F03BDF00D0000C030E9B5F0AE374
:10149000EA6A9B0EE96EEF5005E002D000D0000032
:1014A000EF2EFCD75EEF0AF0985199110EE0949060
:1014B0008B70040E9A6FC80E9B6FE7D79A2FFBD7DD
:1014C0009851D8B499079807EFD728EF0EF0A35199
:1014D000016AA25D03E2A2C000F00CD0006A080E0F
:1014E000A46FA2370036A351005CD8B0006E01365D
:1014F000A42FF7D7000C0150A0C0A2F0640EA36F78
:10150000E6DF00C0A0F00150300E07E1A1A30CD02F
:10151000A1B70AD0A1B9200E03D0A197A199A181AA
:10152000012601C0A2F08FDFA0C0A2F00A0EA36FB7
:10153000CEDF00C0A0F00150300E06E1A1B708D008
:10154000A1A106D0A1B9200E012601C0A2F07BDF27
:10155000300EA027A0C0A2F076DF000CB60E006E01
:10156000036A026A016AA451A511A611A71102E13A
:10157000006A0DD0D89001BE09D0A437A537A63790
:10158000A737033602360136002EF4D7019E000C31
:10159000A451D8B4A5D0B06FA851D8B4A1D0B05F31
:1015A00005E37F0EB027D8B09BD006D0810EB05F88
:1015B000D8A096D0D8B494D0B0C000F0016A026A26
:1015C000036AAF6BA5C0AEF0AE8FA6C0ADF0A7C0EA
:1015D000ACF0190EB06FAB51AC5F0DE2010EAD5F18
:1015E0000AE2AE5F08E2AF5F06E2AF2BAE2BAD2B97
:1015F000AB51AC2728D0AA51AD5F12E2010EAE5F0D
:101600000FE2AF5F0DE2AF2BAE2BAA51AD27AB516E
:10161000AC2719E3AD2B17E1AE2B15E1AF2B13D09F
:10162000A9518009AE5F0EE2010EAF5F0BE2AF2B56
:10163000A9518009AE27AA51AD27E9E3AE2BE7E116
:10164000AF2BE5D70380B02F01D00BD0D890AC37AB
:10165000AD37AE37AF37D890033602360136B137E3
:10166000BAD7B1A106D0D890013202320332B133D9
:1016700002D0000635E0B1BF1ED0D890AC37AD37F0
:10168000AE37AF37AB51AC5F07E2010EAD5F04E29E
:10169000AE5F02E2AF5F1AE3AA51AD5F05E2010E51
:1016A000AE5F02E2AF5F12E3A9518009AE5F03E2D1
:1016B000010EAF5F0BE3032A09E1022A07E1012AC9
:1016C00005E1002A0DE0013202320332A5C0B0F07C
:1016D000A951B01BB0AF02D0018E06D0019E04D03C
:1016E000006A016A026A036A000CB791F2BEB78110
:1016F000F29E90513F0802E23F0E906F9051902B66
:10170000036A500FE96E000E0320EA6EB6C0EFFFC9
:10171000F29EB7B1F28E186AF2BE188EF29E020ED9
:10172000DC6F5FEC06F018BEF28E015207E0186A1B
:10173000F2BE188EF29E2FDC18BEF28EBAEF0BF0BE
:1017400090513F0814E2186AF2BE188EF29E020E03
:10175000DC6F5FEC06F018BEF28E015207E0186AEB
:10176000F2BE188EF29E17DC18BEF28EE9D7B5C015
:10177000B6F0BBD7000C006A016A026A036ABD6B4F
:10178000BE6BBF6BC06BBC51BB11BA11B9112CE061
:10179000200EC16FD890B537B637B737B837BD37D9
:1017A000BE37BF37C037BC51C05D08E1BB51BF5D1C
:1017B00005E1BA51BE5D02E1B951BD5D0FE3B9511A
:1017C000BD5FBA51D8A0BA3DBE5FBB51D8A0BB3DEA
:1017D000BF5FBC51D8A0BC3DC05FD8800036013689
:1017E00002360336C12FD6D7EA6ABD0EE96E000C69
:1017F000E950AC6F3B0EB36F9A0EB26FCA0EB16F69
:10180000B06B0A0EAE6FABC0B8F0AAC0B7F0A9C0FB
:10181000B6F0A8C0B5F0B3C0BCF0B2C0BBF0B1C068
:10182000BAF0B0C0B9F0A7DF0150EFCFA8F0ECCF0D
:10183000A9F0ECCFAAF0ECCFABF000520FE1AE5123
:10184000010A0CE0AC510BE00F0BAE5D01E00CE2C5
:10185000ACBF0AD0ACBD03D0200E02D0AC6B300EB2
:10186000002600C0B5F06CDFB3C0B8F0B2C0B7F06E
:10187000B1C0B6F0B0C0B5F0BC6BBB6BBA6B0A0EB2
:10188000B96F79DF03C0B3F002C0B2F001C0B1F0AC
:1018900000C0B0F0AE2FB7D73AEF10F0B551D8B4C2
:1018A00071D0006EB951D8B46DD0002604E3810E1A
:1018B000002668E204D07F0E005E64E363E0B6C0F9
:1018C000BDF0BA51BD1BB68FBA8FB851BC03F4CF6F
:1018D000BFF0B751BB03F4CF03F0F3CFBEF0BC03AE
:1018E000F350BF27F450BE23000E0322B851BB03B0
:1018F000F350BF27F450BE23000E026A03220222D7
:10190000B651BC03F350BE27F4500322000E02224E
:10191000B651BB03F3500326F4500222000E016AB5
:101920000122B851BA03F350BE27F4500322000E2F
:1019300002220122B751BA03F3500326F4500222C7
:10194000000E0122B651BA03F3500226F4500122D0
:10195000002A01BE05D0BE37033602360136000626
:10196000000EBEAF0AD0032A02220122015005E177
:10197000025003E1035001E1002ABDBF018EBDAF5B
:10198000019E04D0006A016A026A036AFCEF0CF04F
:10199000B551B608B56F036AB6C0B9F0B68FD89026
:1019A000B633B733B8330332023201320032B52FC7
:1019B000F6D7B9AF0BD0001E011E021E031E002A6F
:1019C000D8B4012AD8B4022AD8B4032A0FEF0DF0F4
:1019D000E950AD6FAC51AF6F19E0ABC0B8F0AAC021
:1019E000B7F0A9C0B6F0A8C0B5F0BC6BBB6B200EB9
:1019F000BA6F820EB96F52D703C0ABF002C0AAF023
:101A000001C0A9F000C0A8F0AF2FE7D7ABC0B8F075
:101A1000AAC0B7F0A9C0B6F0A8C0B5F0B9D703C046
:101A2000ABF002C0AAF001C0A9F000C0A8F0ABAFB3
:101A30000DD0AD07AD8BA81FA91FAA1FAB1FA82BE8
:101A4000D8B4A92BD8B4AA2BD8B4AB2B3B0EB46F07
:101A50009A0EB36FCA0EB26FB16B0A0EAF6FAC5174
:101A6000D8B4AD2BABC0B8F0AAC0B7F0A9C0B6F0DF
:101A7000A8C0B5F0B4C0BCF0B3C0BBF0B2C0BAF0FF
:101A8000B1C0B9F078DE0150EFCFA8F0ECCFA9F0EB
:101A9000ECCFAAF0ECCFABF000520FE1AC29AF5D78
:101AA0000CE0AD510CE00F0BAF5D01E037E2ADBFD4
:101AB00035D0ADBD04D0200E2DD0200EAD17ADAB6E
:101AC0000CD0AD9BAC51D8A4AD070050AD6F2D0E1E
:101AD000B56F36DEAD51006EAD6BAC51AF5D0AE156
:101AE0000050AD6F2E0EB56F2BDEAD51006E200E87
:101AF000AD17000E300EADAB0DD0AD9BAC51D8A4E0
:101B0000AD070050AD6F2D0EB56F1ADEAD51006EF2
:101B1000AD6B300E002600C0B5F012DEB4C0B8F0D8
:101B2000B3C0B7F0B2C0B6F0B1C0B5F0BC6BBB6B20
:101B3000BA6B0A0EB96F1FDE03C0B4F002C0B3F077
:101B400001C0B2F000C0B1F0AF2F8CD7000CF86A22
:101B5000D09E088EEA6AE96AC150C00B0F09C16EB7
:101B6000070EB46E356A040E366E0C0E376E386A88
:101B70003C6A906B976BC150C00B0F09C16EF19E10
:101B8000C290B098C69A949E93809392010EC66EAE
:101B9000000EC76ED190870ED56ECD6A000ECA6E4C
:101BA000000ECB6EB16A070EB46E9250926E130E99
:101BB000006E002EFED700D0B450A19CB56AF28A08
:101BC000C00EF2129EEF09F026D4010EA36FA46F8F
:101BD00029DC986B98511EEC01F0982B006EA26FD7
:101BE00032DC0E0E985DF6E1010EA36F020EA46FBB
:101BF00019DC986B985133EC01F0982B006EA26FB2
:101C000022DC0C0E985DF6E1040E986FFA0EA36FBD
:101C1000F7EC08F0982FFAD7986B985147EC01F041
:101C2000982B006EA26F0FDC130E985DF6E194A165
:101C3000FED7986B98515EEC01F0982B006EA26F66
:101C400002DC110E985DF6E1996B0A0E986F2CD4A8
:101C5000306A2F6A2E6A2D6A94A14DD2010E2D266C
:101C6000D8B02E2AD8B42F2AD8B4302A1C6A1B6ABE
:101C70001A6A196A206A1F6A1E6A1D6A246A236A20
:101C8000226A216A286A276A266A256A986B98510F
:101C900074EC01F0982B006EA26F23EC0AF0120E88
:101CA000985DF5E1958083A09DD0958683B699D007
:101CB000986B98518BEC01F0982B006EA26F23EC7F
:101CC0000AF00D0E985DF5E1958483A47ED0010E97
:101CD000A36FA46F12EC0AF09380000E81B0010E86
:101CE000986F9382000E81B2010E996F9384000E5B
:101CF00081B4010E9A6F9386000E81B6010E9B6F20
:101D00009388000E81B8010E9C6F938A000E81BAF1
:101D1000010E9D6F938C000E81BC010E9E6F938E01
:101D2000000E81BE010E9F6F98C0A0F0180EA16F2B
:101D30007BEC0AF0200EA26F23EC0AF099C0A0F011
:101D4000180EA16F7BEC0AF0200EA26F23EC0AF0B4
:101D50009AC0A0F0180EA16F7BEC0AF0200EA26FC3
:101D600023EC0AF09BC0A0F0180EA16F7BEC0AF0E8
:101D7000200EA26F23EC0AF09CC0A0F0180EA16FF9
:101D80007BEC0AF0200EA26F23EC0AF09DC0A0F0BD
:101D9000180EA16F7BEC0AF0200EA26F23EC0AF064
:101DA0009EC0A0F0180EA16F7BEC0AF0200EA26F6F
:101DB00023EC0AF09FC0A0F0180EA16F7BEC0AF094
:101DC000640EA36FF7EC08F07FD7986B985174EC12
:101DD00001F0982B006EA26F23EC0AF0120E985DB2
:101DE000F5E160D7986B98519FEC01F0982B006E4D
:101DF000A26F23EC0AF0090E985DF5E1938081B0A3
:101E000003D0958283B2FAD72C6A2B6A2A6A296A90
:101E1000D76AD66A938281B218D0958283A215D0F0
:101E20002AC09CF029C09BF0996B9A6BD650D7CFF3
:101E300003F09925196ED7509A211A6E000E2920A9
:101E40001B6E000E2A201C6EE5D7938481B403D04C
:101E5000958283B2FAD72C6A2B6A2A6A296AD76AD2
:101E6000D66A938681B618D0958283A215D02AC0EF
:101E70009CF029C09BF0996B9A6BD650D7CF03F09A
:101E800099251D6ED7509A211E6E000E29201F6EB7
:101E9000000E2A20206EE5D7938881B803D0958262
:101EA00083B2FAD72C6A2B6A2A6A296AD76AD66A59
:101EB000938A81BA18D0958283A215D02AC09CF04B
:101EC00029C09BF0996B9A6BD650D7CF03F0992518
:101ED000216ED7509A21226E000E2920236E000E0B
:101EE0002A20246EE5D7938C81BC03D0958283B2DF
:101EF000FAD72C6A2B6A2A6A296AD76AD66A938E1D
:101F000081BE18D0958283A215D02AC09CF029C02A
:101F10009BF0996B9A6BD650D7CF03F09925256E1D
:101F2000D7509A21266E000E2920276E000E2A20F7
:101F3000286EE5D71CC0A7F01BC0A6F01AC0A5F0FC
:101F400019C0A4F0AEEC0AF003C0A7F002C0A6F0DE
:101F500001C0A5F000C0A4F0AB6BAA6B7A0EA96F0C
:101F6000820EA86FC8EC0AF000C098F001C099F08A
:101F700002C09AF003C09BF020C0A7F01FC0A6F0DB
:101F80001EC0A5F01DC0A4F0AEEC0AF003C0A7F07F
:101F900002C0A6F001C0A5F000C0A4F0AB6BAA6B14
:101FA0007A0EA96F820EA86FC8EC0AF000C09CF0F0
:101FB00001C09DF002C09EF003C09FF024C0A7F0B6
:101FC00023C0A6F022C0A5F021C0A4F0AEEC0AF018
:101FD00003C0A7F002C0A6F001C0A5F000C0A4F0A5
:101FE000AB6BAA6B7A0EA96F820EA86FC8EC0AF0D1
:101FF00000C0A0F001C0A1F002C0A2F003C0A3F095
:1020000028C0A7F027C0A6F026C0A5F025C0A4F0E0
:10201000AEEC0AF003C0A7F002C0A6F001C0A5F024
:1020200000C0A4F0AB6BAA6B7A0EA96F820EA86FEA
:10203000C8EC0AF000C0A4F001C0A5F002C0A6F0F0
:1020400003C0A7F00A0EB56FA0EC0BF00D0EB56F34
:10205000A0EC0BF0200EB56FA0EC0BF0070EE96EB4
:1020600030C0ABF02FC0AAF02EC0A9F02DC0A8F050
:10207000F8EF0BF0200EB56FA0EC0BF0060EE96E3A
:102080009BC0ABF09AC0AAF099C0A9F098C0A8F084
:10209000AC6B9EDC200EB56FA0EC0BF0060EE96E6B
:1020A0009FC0ABF09EC0AAF09DC0A9F09CC0A8F054
:1020B000AC6B8EDC200EB56FA0EC0BF0060EE96E5B
:1020C000A3C0ABF0A2C0AAF0A1C0A9F0A0C0A8F024
:1020D000AC6B7EDC200EB56FA0EC0BF0060EE96E4B
:1020E000A7C0ABF0A6C0AAF0A5C0A9F0A4C0A8F0F4
:0A20F000AC6B6EDCB1D590D5030097
:020000040030CA
:0E0000003CCE390E0005A1000FC00FE00F40EE
:00000001FF
